:06000000020DF002006B8E
:03000B0002006B85
:0300130002006B7D
:03001B0002006B75
:0300230002006B6D
:03002B0002006B65
:0300330002006B5D
:03003B0002006B55
:0300430002006B4D
:03004B0002006B45
:0300530002006B3D
:03005B0002006B35
:0300630002006B2D
:01006B003262
:1000800002006B0002006B0002006B0002006B00BC
:1000900002006B0002006B0002006B0002006B00AC
:1000A00002006B0002006B0002006B0002006B009C
:0800B00002006B0002006B006E
:1001000002006B0002006B0002006B0002006B003B
:1001100002006B0002006B0002006B0002006B002B
:1001200002006B0002006B0002006B0002006B001B
:1001300002006B0002006B0002006B0002006B000B
:1001400002006B0002006B0002006B0002006B00FB
:1001500002006B0002006B0002006B0002006B00EB
:1001600002006B0002006B0002006B0002006B00DB
:1001700002006B0002006B0002006B0002006B00CB
:030DF600020DFEED
:030E1100020DF9D6
:050DF9001204BA80FEA7
:10018000C200E4F508F509F50AD201750B00750CFB
:100190000012069F12069C75CB6375CAC0758E004F
:1001A00075C804D2AFD2B0D2B190E60B7403F000A0
:1001B00090E61074A0F00090E61174A0F00090E6B4
:1001C0001274A2F00090E61474E3F00090E6157447
:1001D000A0F00090E6137420F00090E6047480F024
:1001E0000090E6047482F00090E6047484F00090BD
:1001F000E6047486F00090E6047488F00090E6044B
:10020000E4F00090E6497482F00090E6497482F0D0
:100210000090E6497488F00090E6497488F00090F8
:10022000E60BE4F00090E618E4F00090E619E4F044
:100230000090E61A7408F00090E61B7410F000902D
:10024000E6267402F00090E627E4F00090E60274DF
:10025000EBF00043B0100022AA82850C827583E087
:10026000EAF0050C0509E4B50902050A22C01AE501
:1002700081F51A2404F58120000302043512069B3F
:1002800090E6A2E0FA30E103020311E509450A60B5
:10029000687AC07BE78B9D7AC07BE77B008A9E9063
:1002A000E67C7431F07460F0C3743E9509E4950AFD
:1002B00050107A3EE50924C2F509E50A34FFF50A33
:1002C0008007AA09E4F509F50A8A037C007DE08D20
:1002D0009A850B9B8A041AEC601090E67BE090E60E
:1002E0007CF07C007DE08D9A80EA859B0B0090E697
:1002F0008F74022BF0D2CF801830CF1590E7C074E6
:1003000031F090E7C17460F00090E68F7402F0C2A3
:10031000CFE5AA30E003020435C3E50994C1E50A3C
:100320009400400302043590E690E0FB7A0090E6EA
:1003300091E07D004202ED4203A81A080808A602D7
:1003400008A6037C007DF08D9A7C007DF07D008CFA
:100350009BA81A08E4F608F6A81A08A91A090909B8
:10036000C3E69708E60997400302042EE5087003E8
:100370000203F6A81A080808A91A09E6C397FE0896
:10038000E60997FFAA087B00C3EA9EEB9F50048A08
:10039000068B078E02E508C39AF508A81A08EE2610
:1003A000F6EF0836F63001248E028F038A048B059F
:1003B0001ABAFF011BEC4D609F90E67BE0F582C00E
:1003C00002C0031206E3D003D00280E08E028F0346
:1003D0008A048B051ABAFF011BEC4D700302035807
:1003E00090E67BE0F582C002C0031207201202589B
:1003F000D003D00280DA90E67BE0FA23235401FB9D
:10040000B401009201EA30E707743F5AF508801200
:100410003001078A821206B980088A821206D51234
:100420000258A81A0806B6000208060203580090EF
:10043000E6917480F0851A81D01A2290E6B8E0FA2D
:1004400020E70C90E6B9E07002D20075820122909C
:10045000E6B9E0FABA902B90E6BCE025E0547FFACA
:100460002400F582E43418F583E0FB90E740F0EADD
:10047000042400F582E43418F583E0FA90E741F0B3
:10048000800C90E7407436F090E7417483F090E67A
:100490008AE4F090E6BEE0FABA0200500790E6BEA9
:1004A000E0FA80027A0290E68BEAF075820122304F
:1004B000020312095312026D80F5C2AF12018012BD
:1004C0000516120D231208BDD2AF1207B20204AFF7
:10E100001201100100000040FB090160000401023F
:10E1100003010A061001FFFFFF400100090237005A
:10E12000020100804B0904000002FFFFFF02070507
:10E1300081024000000705020240000009040100BE
:10E1400002FFFFFF02070586020002000705080222
:03E15000000200CA
:10E154001201100100000040FB09016000040102EB
:10E1640003010A061001FFFFFF4001000902370006
:10E17400020100804B0904000002FFFFFF020705B3
:10E18400810240000007050202400000090401006A
:10E1940002FFFFFF02070586024000000705080290
:10E1A40040000004B0E1B6E1C4E1DCE10603000094
:10E1B40009040E0341006C007400650072006100E4
:10E1C40018035500530042002D0042006C0061000A
:10E1D40073007400650072001203300030003000D8
:0AE1E4003000300030003000300041
:1004D000AA82E50D54FEFBB50D0280298A048C0525
:1004E000E4620EED620FEB2400F582E43418F5832C
:1004F000E0FB7C00620EEC620FE50E33C50F33C5E6
:100500000F92E0F50EAB0D050DEB2400F582E434FF
:1005100018F583EAF022750D00750EAA750FAA75FD
:1005200082001204D07582001204D07A00C3EA64FB
:100530008094865017EA2408F582E434E1F583E0DC
:10054000F582C0021204D0D0020A80E17A00C3EA28
:10055000648094825017EA2423F582E434E1F58321
:10056000E0F582C0021204D0D0020A80E175821C3C
:100570001204D07582001204D07A00C3EA64809419
:10058000825017EA2402F582E434E1F583E0F58233
:10059000C0021204D0D0020A80E17486250DFAF55B
:1005A00082C0021204D090E1B6E0F5821204D0D0ED
:1005B0000290E1B6E02AFAF582C0021204D090E17E
:1005C000C4E0F5821204D0D00290E1C4E02AF582A2
:1005D0001204D090E1DCE0F5821204D07A0090E1C0
:1005E000B6E0FBC3EA64808BF063F08095F05017AF
:1005F000EA24B6F582E434E1F583E0F582C0021224
:1006000004D0D0020A80D77A0090E1C4E0FBC3EAAC
:1006100064808BF063F08095F05017EA24C4F58273
:10062000E434E1F583E0F582C0021204D0D0020A7E
:1006300080D77A0090E1DCE0FBC3EA64808BF06352
:10064000F08095F05017EA24DCF582E434E1F5837C
:10065000E0F582C0021204D0D0020A80D77A00C32B
:10066000EA648094845017EA240EF582E434E1F5BC
:1006700083E0F582C0021204D0D0020A80E17482C5
:10068000250D40087582001204D080F2AA0E901841
:100690007EEAF0AA0F90187FEAF02222222222900E
:1006A000E6007412F090E60174E3F0AAB574FE5A05
:1006B000F5F0741E45F0F5B522E582FA1392B2EA20
:1006C000A2E192B1EAA2E492B3EAA2E5E433FAB479
:1006D000010092B4221206B9A2B0E433FA74024ABD
:1006E000F58222E5821392B3D2B213C2B292B3D290
:1006F000B213C2B292B3D2B213C2B292B3D2B21395
:10070000C2B292B3D2B213C2B292B3D2B213C2B2D5
:1007100092B3D2B213C2B292B3D2B200C2B2222208
:10072000E582A2B01392B3D2B2C2B2A2B01392B316
:10073000D2B2C2B2A2B01392B3D2B2C2B2A2B013BA
:1007400092B3D2B2C2B2A2B01392B3D2B2C2B2A228
:10075000B01392B3D2B2C2B2A2B01392B3D2B2C2A9
:10076000B2A2B01392B3D2B2C2B2F5822222788082
:10077000E84400600C7901901800E4F0A3D8FCD99B
:10078000FAD083D082F6D8FDC082C0837582002261
:1007900090E6A0E04401F022AA8274805AC4235457
:1007A0001FFB740F5A90E6834BF090E683E04420E1
:1007B000F02290E680E0440AF09000FA120DDF90FB
:1007C000E65D74FFF090E65F74FFF05391EF90E602
:0607D00080E054F7F02266
:060E0B00E478FFF6D8FDBB
:060DF000751000751100F2
:1007D60090E680E0FA30E7267512007513E175148D
:1007E600127515E175161C7517E17518707519E106
:1007F60090E6267402F00090E627E4F000227512D7
:10080600547513E17514667515E17516707517E163
:1008160075181C7519E190E626E4F00090E6277439
:1008260040F000225391EF75A100D20232C021C0E0
:10083600E0C0F0C082C083C002C003C004C005C0CF
:1008460006C007C000C001C0D075D0005391EF7537
:10085600A1001207D6D0D0D001D000D007D006D044
:1008660005D004D003D002D083D082D0F0D0E0D01F
:100876002132C021C0E0C0F0C082C083C002C003E4
:10088600C004C005C006C007C000C001C0D075D0F6
:10089600005391EF75A1001207D6D0D0D001D00039
:1008A600D007D006D005D004D003D002D083D082A2
:1008B600D0F0D0E0D021321207D6751B2A751C085D
:1008C600758200120C7C751B33751C08758210121C
:1008D6000C7C751B78751C08758214120C7C90E6CE
:1008E6005C7431F022E582547FFA24F75004758255
:1008F6000022BA010475820122530201E4BA000102
:1009060004F58222AA82BA010C90E6A1E0FB7C00E3
:100916008B828C8322BA810C90E6A2E0FB7C008B52
:10092600828C832253027FEA700C90E6A0E0FB7C67
:10093600008B828C832290E6A3E0FB7C00EAC31343
:10094600FA7D00EA2BFBED3C8B82F58322C20290F6
:10095600E6B8E0FA530260BA00028028BA200280A4
:100966000DBA4002800EBA60028003020C11120713
:1009760090020C1112043BE5826003020C1112076F
:1009860090020C1190E6B8E0FA530280BA80028019
:1009960003020B1290E6B9E0FABA0003020A8BBA18
:1009A60006028035BA08028008BA0A028017020BCE
:1009B6000C90E740E510F090E68AE4F090E68B7440
:1009C60001F0020C1190E740E511F090E68AE4F0A0
:1009D60090E68B7401F0020C1190E6BBE0FABA01C6
:1009E600028017BA02028038BA03028059BA060298
:1009F600801BBA0702803C020A85AA12AB1390E656
:100A0600B3EBF07B0090E6B4EAF0020C11AA14AB4B
:100A16001590E6B3EBF07B0090E6B4EAF0020C1119
:100A2600AA16AB1790E6B3EBF07B0090E6B4EAF0BB
:100A3600020C11AA18AB1990E6B3EBF07B0090E616
:100A4600B4EAF0020C1190E6BAE0FA90E1A7E0FBF6
:100A5600C3EA9B4006120790020C1190E6BAE075B5
:100A6600F002A424A8F58274E135F0F583E0FAA338
:100A7600E090E6B3F07B0090E6B4EAF0020C1112C7
:100A86000790020C1190E6B8E0FA53021FBA000272
:100A9600800ABA0102801BBA0266802C90E740E405
:100AA600F090E741F090E68AF090E68B7402F0024F
:100AB6000C1190E740E4F090E741F090E68AF09060
:100AC600E68B7402F0020C1190E6BCE0F582120887
:100AD600EBE582602590E6BCE0F58212090AE0FAB1
:100AE60053020190E740EAF090E741E4F090E68A8D
:100AF600F090E68B7402F0020C11120790020C11B2
:100B0600120790020C11120790020C1190E6B9E040
:100B1600FA24F45003020C0EEA2A2A900B257302DB
:100B26000C0E020B5B020BD6020BB7020C0E020C6C
:100B36000E020C0E020C0E020C0E020B49020C0EDB
:100B4600020B5290E6BAE0F510020C1190E6BAE0FC
:100B5600F511020C1190E6B8E0FA53021FBA000232
:100B66008005BA0247800A90E6BAE0120790020CA6
:100B76001190E6BAE0703090E6BCE0F5821208EB20
:100B8600E582602390E6BCE0F58212090AAA82ABF0
:100B960083E0FC5304FE8A828B83ECF090E6BCE093
:100BA600F5821207988064120790805F1207908082
:100BB6005A90E6B8E0FA53021FBA004F90E6BAE040
:100BC600FABA01028005BA02028040120790803B01
:100BD60090E6BAE0FA702C90E6BCE0F5821208EBDB
:100BE600E582601A90E6BCE0F58212090AAA82AB99
:100BF60083E0FC4304018A828B83ECF0800D1207AC
:100C0600908008120790800312079090E6A0E044B7
:100C160080F022AA82BA03004005EA249C500122F1
:100C2600740F5AFBBB03028007740F5AFBBB0B45BC
:100C3600A2AF9203C2AFEA2400F582E43400F58342
:100C46007402F07B0074012AFCE43BFDEC2400F501
:100C560082ED3400F583E51CFCF074022AFAE43BCD
:100C6600FBEA2400F582EB3400F583AA1B7B00EA3D
:100C7600F0A20392AF22E582FA2483500122EA54BD
:100C860003600122A2AF9204C2AFEA2400F582E417
:100C96003401F5837402F07B0074012AFCE43BFD09
:100CA600EC2400F582ED3401F583E51CF074022A8C
:100CB600FAE43BFBEA2400F582EB3401F583AA1B38
:100CC600EAF0A20492AF22AA82BA80004005EA2482
:100CD6004B500122EA5403600122A2AF9205C2AF33
:100CE600EA2480F582E43400F5837402F07B007414
:100CF600012AFCE43BFDEC2480F582ED3400F5830B
:100D0600E51CF074022AFAE43BFBEA2480F582EB48
:100D16003400F583AA1BEAF0A20592AF22C2E8C20C
:100D2600EA751B00751C01758243120C19751B8030
:100D3600751C00758253120C190090E650E4F00001
:100D460090E652E4F00090E654E4F00090E656E4B3
:100D5600F00090E65174FFF00090E65374FFF00047
:100D660090E65574FFF00090E65774FFF00090E6A9
:100D760058E4F090E65974FFF090E65AE4F090E6F5
:100D86005B74FFF090E65CE4F090E65D74FFF09033
:100D9600E65EE4F090E65F74FFF00090E660E4F053
:100DA6000090E66174FFF090E662E4F090E663740A
:100DB600FFF090E665E4F090E668740BF05391AFAF
:100DC600D2E8D2EA2222AA82120DCBDAFB2290FBCB
:100DD60050A3E582458370F922AA82AB83120DD413
:0A0DE6001ABAFF011BEA4B70F42259
:0D0DFE0075812112076EE5826003020DF978
:00000001FF
